:100000000C9434000C9451000C9451000C94510049
:100010000C9451000C9451000C9451000C9451001C
:100020000C9451000C9451000C9451000C9451000C
:100030000C9451000C9451000C942E030C9451001C
:100040000C9451000C9451000C9451000C945100EC
:100050000C9451000C9451000C9451000C945100DC
:100060000C9451000C94510011241FBECFEFD8E026
:10007000DEBFCDBF11E0A0E0B1E0E4E9F7E002C0EF
:1000800005900D92A230B107D9F711E0A2E0B1E0DE
:1000900001C01D92A730B107E1F70E9469030C94DB
:1000A000C8030C9400008CE284B981E58CBD0895EE
:1000B0008EBD0DB407FEFDCF08952A988EBD0DB4F8
:1000C00007FEFDCF6EBD0DB407FEFDCF85B194E0F8
:1000D000892785B908951F93182F81E0612F0E9409
:1000E0005D0082E0612F0E945D0083E0612F0E942D
:1000F0005D0084E0612F0E945D0085E0612F0E9419
:100100005D0086E0612F0E945D0087E0612F0E9404
:100110005D0088E0612F0E945D001F9108958AE0D4
:100120006FE00E945D008BE067E00E945D0089E067
:1001300060E00E945D0080E00E946B008CE061E066
:100140000E945D0008951F93182F83E0612F0E9485
:100150005D0084E0612F0E945D0085E0612F0E94B8
:100160005D0086E0612F0E945D0087E0612F0E94A4
:100170005D0088E0612F0E945D001F9108951F932C
:10018000182F81E0612F0E945D0082E0612F0E94A4
:100190005D001F91089581E06FEF0E945D0082E095
:1001A0006FEF0E945D0083E06FEF0E945D0084E0CE
:1001B0006FEF0E945D0085E06FEF0E945D0086E0BA
:1001C0006FEF0E945D0087E06FEF0E945D0088E0A6
:1001D0006FEF0E945D00089581E06FEF0E945D0067
:1001E00082E06FEF0E945D00089581E060E00E9470
:1001F0005D0082E060E00E945D0008951F9380E052
:100200000E94A3008FEF0E94BF00109101018AE0BD
:10021000612F0E945D0088EE93E028EC30E0F90148
:100220003197F1F70197D9F780910601882311F4EE
:10023000115001C01F5F10930101809101018130B5
:1002400019F48093060104C08F3011F41092060156
:100250001F910895AF92BF92CF92DF92EF92FF92DB
:100260000F931F93CF93DF938AE06FE00E945D00AE
:1002700080E00E946B0011E021E0A22EB12C90E3FF
:10028000C92E95E7D92E88ECE82EF12C20C0C501A7
:100290000C2E02C0880F991F0A94E2F7080F812FD5
:1002A000602F0E945D00133040F482EC91E0F70172
:1002B0003197F1F70197D9F703C0C6010197F1F71C
:1002C0002196C830D10519F71F5F193021F000E0E1
:1002D000C0E0D0E0DCCF84EC99E028EC30E0F9011C
:1002E0003197F1F70197D9F7DF91CF911F910F91D6
:1002F000FF90EF90DF90CF90BF90AF900895CF9296
:10030000DF92EF92FF920F931F93CF93DF938AE0D8
:100310006FE00E945D008FEF0E946B0008E041E0FB
:10032000C42ED12C30E3E32E35E7F32E17C0C601DF
:100330000C2E02C0880F991F0A94E2F7181B802F19
:10034000612F0E945D00C7010197F1F721978FEFA0
:10035000CF3FD80761F70150023021F01FEFC7E00F
:10036000D0E0E5CF84EC99E028EC30E0F90131975A
:10037000F1F70197D9F7DF91CF911F910F91FF907E
:10038000EF90DF90CF900895CF92DF92EF92FF929F
:100390001F93CF93DF938AE06FE00E945D0080E0BF
:1003A0000E946B0010E0C0E0D0E0E1E0CE2ED12C46
:1003B00078ECE72EF12CC6010C2E02C0880F991F95
:1003C0000A94E2F7180F81E0612F0E945D0084EC2F
:1003D00099E0F7013197F1F70197D9F72196C830E5
:1003E000D10549F710E0C0E0D0E061E0C62ED12C85
:1003F00058ECE52EF12CC6010C2E02C0880F991F77
:100400000A94E2F7180F82E0612F0E945D0084ECED
:1004100099E0F7013197F1F70197D9F72196C830A4
:10042000D10549F7DF91CF911F91FF90EF90DF90B9
:10043000CF900895CF92DF92EF92FF921F93CF93C8
:10044000DF938AE06FE00E945D008FEF0E946B00F7
:100450001FEFC0E0D0E081E0C82ED12CB8ECEB2E2D
:10046000F12CC6010C2E02C0880F991F0A94E2F7E6
:10047000181B81E0612F0E945D0084EC99E0F70178
:100480003197F1F70197D9F72196C830D10549F78F
:100490001FEFC0E0D0E0A1E0CA2ED12CF8ECEF2E87
:1004A000F12CC6010C2E02C0880F991F0A94E2F7A6
:1004B000181B82E0612F0E945D0084EC99E0F70137
:1004C0003197F1F70197D9F72196C830D10549F74F
:1004D000DF91CF911F91FF90EF90DF90CF90089523
:1004E000CF92DF92EF92FF921F93CF93DF9380E042
:1004F0000E946B0011E021E0C22ED12C98ECE92E75
:10050000F12C18C0B6010C2E02C0660F771F0A949A
:10051000E2F7812F0E945D0084EF91E0F7013197AF
:10052000F1F70197D9F72196C830D10559F71F5F28
:10053000193019F0C0E0D0E0E5CFDF91CF911F91E5
:10054000FF90EF90DF90CF9008951F9310910501D9
:10055000133061F0143018F4113071F405C0153007
:1005600039F0173049F406C083E307C086E605C0BA
:100570008CEC03C089E901C08FEF0E94A30080E6E4
:100580009AEE0197F1F7812F8F5F809305018830F4
:1005900010F0109205011F9108951F93109104010E
:1005A0001F30F1F1103190F41730D1F1183038F4D8
:1005B000133001F1153001F1113091F519C01B30E4
:1005C000F9F01D30F9F0193059F518C0173141F123
:1005D000183138F41331D1F01531D1F0113101F562
:1005E00013C01B31C9F01D31C9F01931C9F412C053
:1005F00088E817C08CEC15C08EEE13C084E411C0DF
:1006000086E60FC087E70DC082E20BC083E309C016
:100610008BEB07C081E105C089E903C08DED01C006
:100620008FEF0E94A30080E29EE40197F1F7812FF3
:100630008F5F809304018F3110F0109204011F919D
:1006400008958BB183608BB90895789482E080938C
:100650006E008CE085BD8EEF87BD08951F920F92CE
:100660000FB60F9211248F9380910201882359F5C0
:1006700080910301882339F580910001813021F0B8
:1006800080910001823039F4499B05C081E080935C
:1006900002011092000180910001882321F08091D5
:1006A0000001823039F4499905C081E0809302014C
:1006B0008093000180910201882329F4489903C0A6
:1006C00081E0809303018F910F900FBE0F901F90D8
:1006D0001895FF920F931F93CF93DF938BB1836095
:1006E0008BB98CE284B981E58CBD0E948F0078942F
:1006F00082E080936E008CE085BD8EEF87BD88E838
:1007000093E128EC30E0F9013197F1F70197D9F73F
:1007100000E0C8ECD0E01091000180910201F0905F
:100720000301813079F4113081F5F8940E94C401FD
:1007300010920201789406C0F8940E942A01109247
:100740000201789481E0F816B1F4F8941092030154
:1007500088EE93E0FE013197F1F70197D9F7112365
:1007600049F4002321F40E947F0101E003C00E94AC
:100770002A0100E07894113029F0002319F40E9436
:10078000A502C9CF0E94FE00C6CF1123D9F6D4CF4F
:04079000F894FFCF0B
:02079400020F52
:00000001FF
